:1000000008308A005E2900008A1D0A128A190A1621
:100010008A11831A0F28A500030EA6001428831244
:10002000A500030EA600A6140A08AD00A50E04083C
:10003000A7002008A8002108A9002208AA00230878
:10004000AB002408AC0083128B1E28280B1946280D
:100050008C308400001C2E280C18482827088400A7
:100060002808A0002908A1002A08A2002B08A30044
:100070002C08A4002D088A000A1A8A150A12260ED6
:1000800083008312250EA618831609008A115528AD
:100090008A115D280A108A100A11820741346C34D3
:1000A0006934763465340A340034B60B5A28B50AFC
:1000B0003C30B6000B118A112E28B10A0319B20A7E
:1000C0000C108A112E2883168511831285111308AE
:1000D00002309300831614186F2883126A28831243
:1000E00013086F0893008316141878288312732856
:1000F0008312130870089300831614188128831242
:100100007C2885118312851500340F30EF00903064
:10011000F00063202A30EF000330F0006320293024
:10012000EF00D030F00063202830EF000230F00004
:1001300063203030EF000230F00063204030EF00E9
:100140000230F00063205030EF000230F0006320F6
:100150000D30EF00F00163206030EF002030F00040
:1001600063202030EF00FF30F00063202130EF00EB
:10017000E030F0006320EF014830F00063200130F0
:10018000EF00F00163200430EF00F0016320053040
:10019000EF00F00163207030EF002230F0006320A8
:1001A0002430EF00FF30F00063202530EF00E03016
:1001B000F00063200830EF000230F00063200930C7
:1001C000EF00F00163200C30EF000F30F0006320EF
:1001D0002B30EF00F00163200F30EF00F0016320BF
:1001E0003130EF000830F00063203230EF00F001D2
:1001F00063203530EF000630F00063204130EF001F
:100200000830F00063204230EF00F00163204530F9
:10021000EF000630F00063205130EF000830F000AE
:1002200063205230EF00F00163205530EF000630BC
:10023000F00063208A1576298511831685118312B3
:100240001308A03093008316141828298312232939
:1002500083121308930183161418302983122B2953
:1002600083121308EF0085158316851183126F081A
:10027000A100003485118316851183121308033001
:1002800093008316141846298312412983121308F8
:100290006F089300831614184F2983124A2983127A
:1002A00013089301831614185729831252298312B5
:1002B0001308F00085158316851183127008A100BC
:1002C00000341C212108ED006D1C9E296630EF00D2
:1002D0003A21A108031D6C296730EF003A2121085B
:1002E000EE006E08C0390038031D9E295130EF0022
:1002F0000830F00063205230EF00F00163205530E9
:10030000EF000630F00063203630EF006630F0007A
:1003100063203730EF006E08F00063203830EF00C4
:10032000F00163203930EF00F00163203A30EF0034
:10033000F00163203B30EF00F00163202C30EF0030
:10034000F00163208A15A529851183168511831272
:1003500013088130930083161418B0298312AB2937
:10036000831285158316851183128A153E2A8E30D5
:10037000A0006E08A1006D08A200A301A108031D42
:10038000CB292208A100A2010830A002A108031D68
:10039000CB29A001D3290310A11BD229A20DA10DA5
:1003A000A003CB29A113000000346D080319462ACD
:1003B000F50071080319462AF507031CE029E7290F
:1003C0007F30F502031C462A0319462AEB298130A7
:1003D000F5070318462A7508A000A101A201A30190
:1003E0006E08F900F9176F08F8007008F700183068
:1003F000F500F601771C142A7408A307031C062ACB
:10040000A20A031D062AA10A0319F6177308A207F8
:10041000031C0D2AA10A0319F6177208EF00EF1743
:100420006F08A1070318F617F60DA10CA20CA30C78
:10043000F90CF80CF70C0310F50BF9290130A007A3
:100440000318462AA11B2B2AF90DA30DA20DA10DFD
:10045000A0030319462AF91F3C2AA30A031D3C2ABC
:10046000A20A031D3C2AA10A031D3C2AA10CA20CCE
:10047000A30CA00A0319462A6E08F6007208F606B5
:10048000F61F442AA1174A2AA1134A2AA001A10152
:10049000A201A30100008A15732B80300418F20614
:1004A000F7016E08F6007208F6066D0803193C2B7A
:1004B000F5007508A00071080319452BF502031912
:1004C000E22A0318642AA02A7208FB00FB177308AB
:1004D000FA007408F900F8010310FB0CFA0CF90C8F
:1004E000F80CF50B6B2AF61F782A7714592B771026
:1004F00075107716703084006E2B7712F61B8A2ADF
:10050000751C952AFB0CFA0CF90CF80CA00A0319BF
:10051000542B952AFB1B982A0310F80DF90DFA0DA0
:10052000FB0DA0030319542B8A2A7717012B77138D
:100530006E08F600F61F9E2AFB174D2BFB134D2B62
:100540007108F5007508A0006D08F5026E08FB0043
:10055000FB176F08FA007008F900F8010310FB0C94
:10056000FA0CF90CF80CF50BAD2AF61FBA2AF714A1
:10057000592BF7107510F716743084006E2BF71294
:10058000F61BCC2A751CD72AFB0CFA0CF90CF80CBC
:10059000A00A0319542BD72AFB1BDA2A0310F80DE3
:1005A000F90DFA0DFB0DA0030319542BCC2AF717F4
:1005B000012BF7137208F600F61FE02AFB174D2BEC
:1005C000FB134D2B7208FB00FB177308FA0074082D
:1005D000F900F61FEF2AFB137715592B7711F80155
:1005E0007510703084006E2BF61B172B6E08F6000A
:1005F000751C012BFB0CFA0CF90CF80CA00A031962
:10060000542BF81F122BF90A031D122BFA0A031D93
:10061000122BFB0A031D122BFB0CFA0CF90CA00A7F
:100620000319542B771B972AF71BD92A362B8030B6
:10063000FB06FB1F1F2B592B7208F6002C2B6E0894
:10064000F600FB08031D2C2BFA08031D2C2BF908C0
:10065000031D2C2BA0014D2BFB1B362B0310F80D7B
:10066000F90DFA0DFB0DA00B2C2B542BF61F3A2B7A
:10067000FB174D2BFB134D2B7108A0007208FB00DC
:100680007308FA007408F9004D2B6D08A0006E087D
:10069000FB006F08FA007008F9007B08A1007A08D7
:1006A000A2007908A3008D2BA001A101A201A30142
:1006B0008D2BF909FA09FB09F809F80A031D672BC4
:1006C000F90A031D672BFA0A031D672BFB0A77182B
:1006D000772AF718B92A7719EE2A1C2B0008F90790
:1006E000031C782BFA0A031D782BFB0A03197514D7
:1006F00084030008FA07031C802BFB0A03197514F6
:1007000084030008801B852B803AFB0703187514AF
:10071000771A7D2AF71ABF2AF42A00008A15872B38
:100720007008A1016F020318982B6F08A000A42B7A
:10073000A0010830F100EF0DA00D70082002031891
:10074000A000A10DF10B9B2B00346E18C02BEE18EE
:10075000D42B6D08EF006430F00090232008ED00EA
:1007600021083030031DB92B6E19C02BEE19203033
:10077000BB2B6E11EE11A10721080C1EBD2B990099
:100780006D08EF000A30F00090232008ED002108EA
:100790003030031DCF2B6E19D42BEE192030A1075A
:1007A00021080C1ED12B99003030ED076D080C1E6E
:1007B000D72B990000348E30A0006D08A0026E087F
:1007C000A2006F08A100A217A0080319F22B0310C2
:1007D000A208031DEE2BA1080319F22BA20CA10CF9
:1007E000A00BE72B00008A15702C0408F600700E91
:1007F000F038F200F207E23EF300323EF5007008F6
:100800000F39F307F307F507E93EF400F407F4079F
:100810006F0E0F39F407F507F40DF50DF509F50D19
:100820006F080F39F507F20D0730F1000A30F507B0
:10083000F403031C172CF407F303031C1B2CF3070E
:10084000F203031C1F2CF207F103031C232C760870
:10085000840007308405713084070008A000031D60
:10086000372C761A3F2CF619392C20303A2C0830C8
:10087000F6003030A00720080C1E3C2C9900840A9A
:1008800075300402031D2D2C0008A0003030A00795
:1008900020080C1E492C9900003471080319132DEF
:1008A000FD0075080319132DFD020318582C5D2C4B
:1008B0007F30FD070318132D632C8130FD02031CCC
:1008C000132D0319132D7D08A000A101A201A3017E
:1008D000FC017208FB00FB177308FA007408F900AA
:1008E0001930FD007808F9020318862C0130FA024D
:1008F0000318862CFB020318862CFC020318862C96
:10090000FC0AFB0AFA0A7808F907B82C7708FA02F9
:100910000318A12C0130FB020318A12CFC020318C0
:10092000A12CFC0AFB0A7708FA077808F907031CD0
:10093000B82CFA0A031DB82CFB0A031DB82CFC0ABC
:10094000B82C76088038FB020318B72C0130FC0263
:100950000318B72CFC0A76088038FB077708FA07DB
:10096000031C952CFB0A031D952CFC0A952C2314C3
:10097000FD0BBB2CC62C0310F90DFA0DFB0DFC0D65
:100980000310A30DA20DA10DFE0D722C7E1CCE2C0A
:100990000310A10CA20CA30CFE0CD12CA003031974
:1009A000132DFE1BFA2C0310F90DFA0DFB0DFC0D97
:1009B0007808F9020318E62C0130FA020318E62C35
:1009C000FB020318E62CFC02031C092D7708FA022F
:1009D0000318F12C0130FB020318F12CFC02031C5C
:1009E000092D76088038FB020318FA2C0130FC022E
:1009F000031C092DA30A031D092DA20A031D092D9D
:100A0000A10A031D092DA00A0319132DA10CA20C84
:100A1000A30C7208FD007608FD06FD1F112DA1171D
:100A2000172DA113172DA001A101A201A301000000
:100A3000003404088316A500A6018312F61F242D96
:100A40002D300C1E212D9900F617750803190C2E58
:100A50007F307502031CAE2DF5008316AB01043008
:100A6000AC0083120310F80DF70DF60D8316A60DDA
:100A7000AC0B3B2D3D2D8312322D831204307502B9
:100A800003184E2D03307502031D002E0A30831605
:100A9000260203184D2D8312002E83120330F50217
:100AA0008316AB0A831212270310F80DF70DF60D0B
:100AB0008316A60D8312E82602308316AC0083123B
:100AC00003108316A60C8312F60CF70CF80C831691
:100AD000AC0B6B2D6D2D8312602D83121227043009
:100AE0008316AC00831203108316A70CA80CA90C64
:100AF000AA0CAC0B7C2D7E2D8312732D8312E8265D
:100B0000122783162908AA002808A9002708A80088
:100B1000A7018312E826122783162808AA002708AF
:100B2000A900A701A8018312E8268316A61D9A2D05
:100B300083123E2D8312F508031DA52DF80AF70A2E
:100B4000F60A8316A60A8312002E0310F80DF70D7D
:100B5000F60D8316A60D8312F5033E2DF509F50A51
:100B60007F30F5078316AB010430AC00831203100D
:100B7000F80DF70DF60D8316A60DAC0BC02DC22D8A
:100B80008312B72D04308312F50705307502031C5C
:100B9000102E12270310F80DF70DF60D8316A60D73
:100BA00003108312F80DF70DF60D8316A60D8312B0
:100BB000E8260310F80DF70DF60D8316A60DAB0A07
:100BC0000330AC00831203108316A60C8312F60CBC
:100BD000F70CF80C8316AC0BEE2DF02D8312E32DE1
:100BE00003308312F5028316261AF82D8312C52DC1
:100BF0000310A60C8312F60CF70CF80CF503C52DA8
:100C0000F509F50A0330F50783162B08A100A300A8
:100C1000250AA3078312512E8316250AAB008312DF
:100C200030300C1E112E99008316A508031D1A2EB4
:100C30008312E62E2E3083120C1E1C2E9900831672
:100C40002B08A400A403250824020318292E8312CC
:100C50002C2E2508A40083128316A408031D322E0F
:100C600083123E2E831230300C1E342E99008316D0
:100C7000A40B3B2E3D2E8312332E831283162B089A
:100C8000AC00250AAC02031C472E8312232F8312CB
:100C9000F5038316250AA3002B08A3022308A1004D
:100CA000831283162608A000831275080319642E88
:100CB0008316A200831203108316A00CA20B612ED0
:100CC000632E83125B2E831283162308031D6A2E64
:100CD0008312E62E3030200783120C1E6D2E9900F1
:100CE000831621080319762E8312802EA508031D72
:100CF0007B2E8312E62E2E3083120C1E7D2E990041
:100D00008316A103A303031D872E8312E62E8312ED
:100D100075080319972E8316A200831203108316F9
:100D2000A00DA20B942E962E83128E2E8312831664
:100D30002008A6022608A700831276088316A800BA
:100D4000831277088316A900831278088316AA00F5
:100D500003108312F80DF70DF60D8316A60D031080
:100D60008312F80DF70DF60D8316A60D2A088312CF
:100D7000F807031CC42EF70FC42EF60AF608031D4D
:100D8000C42E8316A60A8312831629088312F70736
:100D9000031CD12EF60AF608031DD12E8316A60ACF
:100DA0008312831628088312F607031CDA2E831693
:100DB000A60A831283162708A60703108312F80DCC
:100DC000F70DF60D8316A60D8312512E0000232F6A
:100DD00083162A088312F807031CF72EF70FF72E45
:100DE000F60AF608031DF72E8316A60A8312831649
:100DF00029088312F707031C042FF60AF608031DBF
:100E0000042F8316A60A8312831628088312F60776
:100E1000031C0D2F8316A60A831283162708A60724
:100E20008312003483162608A700831276088316DF
:100E3000A800831277088316A90083127808831606
:100E4000AA008312003400000034FF3FFF3FFF3F41
:100E5000FF3FFF3FFF3FFF3FFF3FFF3FFF3FFF3FA2
:100E6000FF3FFF3FFF3FFF3FFF3FFF3FFF3FFF3F92
:100E7000FF3FFF3FFF3FFF3FFF3FFF3FFF3FFF3F82
:100E8000FF3FFF3FFF3FFF3FFF3FFF3FFF3FFF3F72
:100E9000FF3FFF3FFF3FFF3FFF3FFF3FFF3FFF3F62
:100EA000FF3FFF3FFF3FFF3FFF3FFF3FFF3FFF3F52
:100EB000FF3FFF3FFF3FFF3FFF3FFF3FFF3FFF3F42
:100EC000FF3FFF3FFF3FFF3FFF3FFF3FFF3FFF3F32
:100ED000FF3FFF3FFF3FFF3FFF3FFF3FFF3FFF3F22
:100EE000FF3FFF3FFF3FFF3FFF3FFF3FFF3FFF3F12
:100EF000FF3FFF3FFF3FFF3FFF3FFF3FFF3FFF3F02
:100F0000FF3FFF3FFF3FFF3FFF3FFF3FFF3FFF3FF1
:100F1000FF3FFF3FFF3FFF3FFF3FFF3FFF3FFF3FE1
:100F2000FF3FFF3FFF3FFF3FFF3FFF3FFF3FFF3FD1
:100F3000FF3FFF3FFF3FFF3FFF3FFF3FFF3FFF3FC1
:100F4000FF3FFF3FFF3FFF3FFF3FFF3FFF3FFF3FB1
:100F5000FF3FFF3FFF3FFF3FFF3FFF3FFF3FFF3FA1
:100F6000FF3FFF3FFF3FFF3FFF3FFF3FFF3FFF3F91
:100F7000FF3FFF3FFF3FFF3FFF3FFF3FFF3FFF3F81
:100F8000FF3FFF3FFF3FFF3FFF3FFF3FFF3FFF3F71
:100F9000FF3FFF3FFF3FFF3FFF3FFF3FFF3FFF3F61
:100FA000FF3FFF3FFF3FFF3FFF3FFF3FFF3FFF3F51
:100FB000FF3FFF3FFF3FFF3FFF3FFF3FFF3FFF3F41
:100FC000FF3FFF3FFF3FFF3FFF3FFF3FFF3FFF3F31
:100FD000FF3FFF3FFF3FFF3FFF3FFF3FFF3FFF3F21
:100FE000FF3FFF3FFF3FFF3FFF3FFF3FFF3FFF3F11
:100FF000FF3FFF3FFF3FFF3FFF3FFF3FFF3FFF3F01
:101000000408F600F701EE1F09282D300C1E0628F3
:101010009900EE176D080319A9287F306D02031C93
:101020006828ED00FC010430FD000310F00DEF0D09
:10103000EE0DF70DFD0B152804306D02031828285E
:1010400003306D02031DA2280A307702031CA22878
:101050000330ED02FC0A52210310F00DEF0DEE0DEE
:10106000F70D39210230FD000310F70CEE0CEF0CE8
:10107000F00CFD0B342852210430FD000310F80C55
:10108000F90CFA0CFB0CFD0B3E28392152217A0891
:10109000FB007908FA007808F900F801392152219B
:1010A0007908FB007808FA00F801F9013921F719ED
:1010B0001C28ED08031D6128F00AEF0AEE0AF70A62
:1010C000A2280310F00DEF0DEE0DF70DED031C2817
:1010D000ED09ED0A7F30ED07FC010430FD0003103F
:1010E000F00DEF0DEE0DF70DFD0B6F280430ED0741
:1010F00005306D02031CB02852210310F00DEF0DD6
:10110000EE0DF70D0310F00DEF0DEE0DF70D39217B
:101110000310F00DEF0DEE0DF70DFC0A0330FD008E
:101120000310F70CEE0CEF0CF00CFD0B90280330C5
:10113000ED02771E78280310F70CEE0CEF0CF00C84
:10114000ED037828ED09ED0A0330ED072B30FD00A3
:10115000B328F701EE01EF01F001FD01FC01B32816
:10116000ED032D30FD00F2017708F1006D08031941
:10117000BE28F3000310F10CF30BBA287608F30035
:1011800072087302031C0B29303071070C1EC6282D
:101190009900F208031DD0282E300C1ECD2899008E
:1011A000F20A6D080319D928F3000310F10DF30BAF
:1011B000D5287108F7027708F8006E08F9006F0863
:1011C000FA007008FB000310F00DEF0DEE0DF70DA7
:1011D0000310F00DEF0DEE0DF70D7B08F007031C6B
:1011E000F728EF0FF728EE0AEE080319F70A7A0836
:1011F000EF07031CFF28EE0AEE080319F70A790827
:10120000EE070318F70A7808F7070310F00DEF0D43
:10121000EE0DF70DB428000045300C1E0D29990085
:101220007D08031916290C1E13299900F4017C0866
:10123000F5000A30F502031C2D29F40AF502031803
:101240001D29F507303074070C1E24299900303011
:1012500075070C1E292999003729F50730300C1E17
:101260002F299900303075070C1E34299900000091
:101270005B297B08F007031C4329EF0F4329EE0A83
:10128000EE080319F70A7A08EF07031C4B29EE0A48
:10129000EE080319F70A7908EE070318F70A780829
:1012A000F70700347708F8006E08F9006F08FA00B5
:1012B0007008FB00003400008A158B2D84011F305C
:1012C00083059F30840007308000333083169900F7
:1012D00022309800903083129800831687120716E8
:1012E00087113030831294008A1185288A15B00145
:1012F000AF01B201B1013C30B60081010730A0005E
:10130000A01D8A2907308101813084000008C0397E
:101310000F3880006400813084000008C039200448
:1013200080008B16073090008C3084000014C03091
:101330008B04B5010514831605108312063035029F
:101340000318A72964008A1161298A159E298E0134
:101350008F018A111C218A152108CF00ED016D082B
:101360008A114A208A15ED0A0C1EB429990006300C
:101370006D02031DAF294F1C8A2A64006630EF00FE
:101380008A113A218A152108D100D108031DC829E4
:1013900064006730EF008A113A218A152108D000D5
:1013A0005008C0390038031DDD290B12B001AF0110
:1013B000B201B1018E018F010B16EE010E08ED0096
:1013C000F0010F08EF006F08A3000001A000230840
:1013D0006E04B00020086D04AF003630EF006630B8
:1013E000F0008A1163208A153830EF002F08F000D2
:1013F0008A1163208A153008ED003930EF006D083E
:10140000F0008A1163208A153A30EF003108F000AD
:101410008A1163208A153208ED003B30EF006D0819
:10142000F0008A1163208A155008C039A0004030AE
:101430002002031D1B2A3530EF000630F0008A1110
:1014400063208A155008033900380319352A5008DB
:101450000339A000013020020319352A500803394E
:10146000A00002302002031D762A3730EF0050081A
:10147000F0008A1163208A158A11A4298A15500860
:1014800003390038031D502A8616831686128312EC
:101490008611831686118312861083168610831296
:1014A00050080339A00001302002031D632A861270
:1014B0008316861283128615831686118312861070
:1014C00083168610831250080339A00002302002D0
:1014D000031D762A861283168612831286118316BE
:1014E0008611831286148316861083125008C03921
:1014F000A00080302002031D842A0B12B001AF012E
:10150000B201B1018E018F012C30EF00F0018A1180
:1015100063208A15CF1C992D7630EF008A113A216D
:101520008A152108D10090305102031DEF2A77302F
:10153000EF008A113A218A152108B7007830EF00B0
:101540008A113A218A152108B8007930EF008A11F2
:101550003A218A152108B9007B30EF008A113A211F
:101560008A15D4012108D3007A30EF008A113A217C
:101570008A15EE012108ED005308A30000016D0754
:10158000A10023080318013E6E07A3002108ED0007
:101590002308EE008A11B7218A152008BA00210815
:1015A000BB002208BC002308BD007D30EF008A117B
:1015B0003A218A15D4012108D3007C30EF008A112A
:1015C0003A218A15EE012108ED005308A30000011D
:1015D0006D07BE0023080318013E6E07BF0091305F
:1015E0005102031D902B7830EF008A113A218A15A1
:1015F000D4012108D3007730EF008A113A218A15EF
:10160000EE012108ED005308A30000016D07C000A2
:1016100023080318013E6E07C1007A30EF008A11DB
:101620003A218A15D4012108D3007930EF008A11BC
:101630003A218A15EE012108ED005308A3000001AC
:101640006D07C20023080318013E6E07C3007C30FB
:10165000EF008A113A218A15D4012108D3007B308A
:10166000EF008A113A218A15EE012108ED00530896
:10167000A30000016D07A10023080318013E6E07B7
:10168000A3002108ED002308EE008A11B7218A1576
:101690002008C4002108C5002208C6002308C7008E
:1016A0007D30EF008A113A218A15EE012108ED0004
:1016B0008A11B7218A152008D5002108D6002208F2
:1016C000D7002308D8005508ED005608EE0057084B
:1016D000EF005808F0008F30F1000030F200F30006
:1016E000F4008A11D5298A1584014408ED004508C3
:1016F000EE004608EF004708F0002008F10021083E
:10170000F2002208F3002308F4008A114D2A8A15FA
:101710002008C4002108C5002208C6002308C7000D
:1017200092305102031D932D7730EF008A113A2138
:101730008A152108C8007830EF008A113A218A15ED
:101740002108C9007930EF008A113A218A15210851
:10175000CA007A30EF008A113A218A152108CB009D
:101760007B30EF008A113A218A152108CC007C30A9
:10177000EF008A113A218A152108CD003230D900B4
:101780003030DA004A08F039A000A00E0F30A00572
:101790002008A00030302007DB004A080F39A000E5
:1017A00030302007DC002F30DD004908F039A00080
:1017B000A00E0F30A0052008A00030302007DE006A
:1017C00049080F39A00030302007DF002F30E0003B
:1017D0004808F039A000A00E0F30A0052008A00096
:1017E00030302007E10048080F39A00030302007D2
:1017F000E2002C30E3004B08F039A000A00E0F30BF
:10180000A0052008A00030302007E4004B080F3965
:10181000A00030302007E5003A30E6004C08F039EF
:10182000A000A00E0F30A0052008A0003030200737
:10183000E7004C080F39A00030302007E8003A30AC
:10184000E9004D08F039A000A00E0F30A0052008D7
:10185000A00030302007EA004D080F39A0003030DA
:101860002007EB00EC01593084000030000403191C
:101870003F2C0C1E392C00089900840A352C2C3082
:101880000C1E402C99003708ED000230EE008A1142
:10189000A5238A152C300C1E4B2C99003808ED001E
:1018A0000230EE008A11A5238A152C300C1E562C0E
:1018B00099003908ED00EE018A11A5238A1501303F
:1018C0003702FC3E03186F2D043E9B2D3A08ED00B5
:1018D0003B08EE003C08EF003D08F0008A11DB2BCE
:1018E0008A152208EE002108ED002C300C1E762C03
:1018F0009900093084006E08F0006D08EF008A112D
:10190000F5238A152E300C1E832C990030300C1EC6
:10191000872C990030300C1E8B2C99003F08EE006C
:101920003E08ED008A11B7218A152008ED00210834
:10193000EE002208EF002308F0006D08F1006E08A9
:10194000F2006F08F3007008F4008830F5007A3078
:10195000F6000030F700F8008A114D248A1520089F
:10196000F1002108F2002208F3002308F4002C30D3
:101970000C1EB82C9900043084007108F500720820
:10198000F6007308F7007408F8008A1119258A1503
:101990004108EE004008ED008A11B7218A152008A1
:1019A000ED002108EE002208EF002308F0006D088A
:1019B000F1006E08F2006F08F3007008F400853043
:1019C000F5004830F6000030F700F8008A114D2489
:1019D0008A152008F1002108F2002208F3002308EC
:1019E000F4002C300C1EF22C990004308400710895
:1019F000F5007208F6007308F7007408F8008A1101
:101A000019258A156F2D3A08F1003B08F2003C08B1
:101A1000F3003D08F4008530F5004830F600003052
:101A2000F700F8008A114D248A152008ED002108DE
:101A3000EE002208EF002308F0002C300C1E1E2DB3
:101A40009900023084006D08F5006E08F6006F08FA
:101A5000F7007008F8008A1119258A153F08EE0072
:101A60003E08ED008A11B7218A152008ED002108F3
:101A7000EE002208EF002308F0002C300C1E3E2D53
:101A80009900043084006D08F5006E08F6006F08B8
:101A9000F7007008F8008A1119258A154108EE0030
:101AA0004008ED008A11B7218A152008ED002108B1
:101AB000EE002208EF002308F0002C300C1E5E2DF3
:101AC0009900043084006D08F5006E08F6006F0878
:101AD000F7007008F8008A1119258A156F2D2C302F
:101AE0000C1E702D9900093084004308F000420854
:101AF000EF008A11F5238A152C300C1E7D2D9900DC
:101B0000043084004408ED004508EE004608EF006C
:101B10004708F00000280A300C1E8C2D99000D306B
:101B20000C1E902D99002C30EF00F0018A116320DB
:101B30008A15A92963000A148A100A158207662CDF
:061B4000662C032D662C4B
:02400E00FA3F77
:00000001FF
